:020000040000FA
:0400000000EF2CF0F1
:0457FC0000000000A9
:1058000097EF2FF000C0E5FF01C0E5FF00EE62F06A
:10581000F9EC2EF0006E00C0F3F000C0F4F0F9ECEB
:105820002EF0006E0001E96F00500001F427F9EC42
:105830002EF0006E0001E86F00500001F427F9EC33
:105840002EF0006E00C0F5F000500001F4270001BA
:10585000F551040A24E10001E951D8A4DBD0E85154
:10586000D8A4D8D00001F351020A01E0D3D0F9EC5A
:105870002EF0006E0001EB6F00500001F427F9ECF0
:105880002EF0006E0001EA6F00500001F427F9ECE1
:105890002EF0006E0001F427F451D8A4B3D000011B
:1058A000F551010A20E1F9EC2EF0006E0001F42719
:1058B000F451D8A4A7D00001F2B3B8EC2DF082ECDB
:1058C0002FF00001F2A50BD0C00E0001E46F570EBF
:1058D000E56FE66BE76BB8EC2DF082EC2FF0590E1C
:1058E00067EC2FF09AD00001EB510001E71914E1A9
:1058F0000001EA510001E6190FE10001E951000140
:10590000E5190AE1C00E0001E815006EC00E0001A5
:10591000E415016E00180FE00001F2A302D0B8EC0C
:105920002DF082EC2FF0E8C0E4F0E9C0E5F0EAC029
:10593000E6F0EBC0E7F00001F551040A01E15ED0AA
:105940000001F551D8A462D00001F351D8B456D06B
:105950000001EB51D8A45AD0EA51E00BD8A456D09C
:105960000001F2A912D00001F35141EC2EF0400EDB
:105970008DEC2FF00001E95141EC2EF00001E851CF
:1059800041EC2EF0200E8DEC2FF0EAC0F8FFE9C0BC
:10599000F7FFE8C0F6FF000100EE6AF022EE00F02B
:1059A000E8513F0BD926D8B0DA2ADD52F9EC2EF0B7
:1059B0000001F427DC6E0900F55C05E00001F283CC
:1059C0002A0E8DEC2FF00001F2A906D0DF5041EC39
:1059D0002EF0200E8DEC2FF00001F32FE7D7F9EC1D
:1059E0002EF0006E0001F427F45108E00001E46994
:1059F000E569E669E7690001F29304D0580E67ECA7
:105A00002FF00BD07A0E67EC2FF007D0750E67ECF5
:105A10002FF003D06C0E67EC2FF0E4CF01F0E4CF51
:105A200000F01200FF0E926E936E946E956E966E5D
:105A3000970ED56E8A809390B06A2F0EAF6EB8869F
:105A4000AC8AAC84AC8CAC90AB8CAB8E0001E46BBC
:105A5000E56BE66BE76B0001E86BE96BEA6BEB6B00
:105A600082EC2FF00001F26B93988A888A90AB98B1
:105A70004B0E8DEC2FF0A1EC2FF00001EC6BED6BD9
:105A80008AB002D0A1EC2FF00001606BB9EC2EF0CF
:105A900000016051D8B45CD08A90AB988AA802D03B
:105AA0008A9801D08A8861C000F00050520A03E150
:105AB00058EC2FF00BD00050500A03E149EC2FF0C6
:105AC00005D00050560A02E175EC2EF00001F2A15B
:105AD0003FD00050450A03E137EC2FF039D0005099
:105AE0003A0A03E102EC2CF033D00050720A03E1D1
:105AF00098EC2EF02DD00050410A03E1C2EC2FF0BB
:105B000027D00050760A24E1006A00016251300A71
:105B100001E1002A0050D880E866D890006A00367B
:105B20000050010BE838E840F46E0001F251F70B29
:105B3000F410F26F320E0001625D006A0036005010
:105B4000010BE838F46E0001F251EF0BF410F26F24
:105B50000001F2B195D70001ED51800F800F02E1F5
:105B6000A10EEC5DD8A08CD7C2EC2FF089D7120023
:105B700000C0E5FF01C0E5FF02C0E5FF03C0E5FF8F
:105B80000001E4513F0B04E0210E8DEC2FF070D0AA
:105B90000001E75103E1E651E00BD8A469D0580EAB
:105BA0000001E55D02E1000EE45D01E361D0E4C0C7
:105BB00000F0E5C001F0E6C002F0E7C003F00050DD
:105BC00001100210031013E100C2E0F001C2E1F085
:105BD00002C2E2F003C2E3F00201006BEF0E016FBC
:105BE0002C0E026FF00E036F0001F28515D00050ED
:105BF000C00A07E10150570A04E1025002E10350D4
:105C000001E00AD0E0C03CF2E1C03DF2E2C03EF269
:105C1000E3C03FF20001F2950001F2A70BD0200E85
:105C20008DEC2FF00001E55141EC2EF00001E45124
:105C300041EC2EF0E6C0F8FFE5C0F7FFE4C0F6FF48
:105C4000940EA9EC2FF00A0002EE00F00001080EFD
:105C5000EE6F080EEF6FEE50F56E0F00EF2FFBD7D3
:105C6000840E77D9EE2FF5D7A694570E67EC2FF058
:105C7000E4CF03F0E4CF02F0E4CF01F0E4CF00F092
:105C8000120000C0E5FF01C0E5FF02C0E5FF006EA5
:105C900000380F0B026E300E02260250016E3A0ED3
:105CA000015C06E30150026E070E02260250016EEF
:105CB00001508DEC2FF00F0E0014006E300E0026F8
:105CC0000050016E3A0E015C06E30150006E070EB3
:105CD00000260050016E01508DEC2FF0E4CF02F051
:105CE000E4CF01F0E4CF00F0120000EE62F000011A
:105CF00060050001EF6FEF07010EEE6FEE51BCEC97
:105D00002FF004E10A0EEE6FBCEC2FF0EE5CD8A48D
:105D10001200EE2BEF2FF2D7EE51BCEC2FF0D8A4EF
:105D20001200560E67EC2FF00001F281F29512007E
:105D300000C0E5FF00EE62F0F9EC2EF0F76EF9EC32
:105D40002EF0F66E720E8DEC2FF0200E8DEC2FF0F3
:105D5000100E006E0900F55041EC2EF0200E8DEC77
:105D60002FF0002EF7D70A0E8DEC2FF0E4CF00F0C5
:105D70001200B6EC2FF0000100EE60F0D9EC2EF02E
:105D8000E86614D0AE50EE6EEE6FEF6FD8B40ED062
:105D9000B6EC2FF0D9EC2EF0E86608D0AE50EE6EDF
:105DA000EF27EE2FF5D7EF53D8B412000001606B48
:105DB00012009EBA08D0F2A4FCD70001EC2B01E33C
:105DC000ED2BE86815D08A98ABB202D0ABA404D012
:105DD000A1EC2FF0E8680CD0ABA009D0AE5005E1E3
:105DE000B6EC2FF0D9EC2EF003D0C2EC2FF0E86A1D
:105DF00012000001EECFEEF0EECFEFF0D00EEE2766
:105E0000EF27F60EEE25F90ED8B0EE27F60EEF25A9
:105E1000F90ED8B0EF27EE39EF25E850120000EE6A
:105E200068F000016051F80F0001EE6F09E0F05DCD
:105E300007E3EE50A86E76EC2FF0A92AEE2FF9D7E3
:105E4000A86A76EC2FF0120000C0E5FF01C0E5FF64
:105E5000006A00EE62F0060E016EEE500026012E82
:105E6000FCD70050E4CF01F0E4CF00F0120000EEC8
:105E700061F0000160510001EE6F07E0EE0705E000
:105E8000EE508DEC2FF0EE2FFBD70A0E8DEC2FF09D
:105E9000120024EC2FF0B80A0AE1010EA96E080ED8
:105EA0000001F06F0FEC2FF0500E67EC2FF0120096
:105EB00024EC2FF0A00A0AE10A0EA96E100E0001D0
:105EC000F06F0FEC2FF0520E67EC2FF0120000C0B5
:105ED000E5FF006E200E8DEC2FF000508DEC2FF0C2
:105EE0000A0E8DEC2FF0E4CF00F01200A69EA69CC7
:105EF000A684550EA76EAA0EA76EA682A6B2FED7DE
:105F0000A69412000001F2930001400EEE6F02EE23
:105F100000F0EE68EE2FFDD7120000C0E5FF006E26
:105F20009EA8FED700C0ADFFE4CF00F0120011EE36
:105F3000FFF021EEFFF0F86AA68EA69C12EC2DF081
:105F4000FFD7ACA2FED78A80AE50AE50AB98AB88DC
:105F50001200A66E550EA76EAA0EA76EA68212009C
:105F6000B2EF2FF012EC2DF0B4EF2FF0FE0ED76E43
:105F7000120ED66EF2941200A96EA69CA69EA68062
:085F8000A8501200FEEF2BF007
:020000040030CA
:0E000000E03ECEE0FF7D9AFFFFFFFFFFFFFF17
:0200000400F00A
:0400000000000000FC
:00000001FF
